:10000000BEC00000F2C00000D6C00000D4C0000096
:10001000D2C00000D0C00000CEC00000CCC00000A4
:10002000CAC00000C8C00000C6C00000C4C00000B4
:10003000C2C00000C0C00000BEC00000BCC00000C4
:100040000C94B110B8C00000B6C00000B4C00000ED
:10005000B2C00000B0C00000AEC00000ACC00000E4
:10006000AAC00000A8C000002E0A370A340A330ACA
:10007000320A310A300A2F0A380A380A380A380A8E
:10008000380A380A380A380A350A380A380A380A63
:10009000380A380A380A380A360A2A035500530043
:1000A0004200200052006500740072006F00500092
:1000B0006100640020004100640061007000740071
:1000C000650072002A037700770077002E00620037
:1000D000720075006E006F006600720065006900B6
:1000E0007400610073002E0063006F006D00040354
:1000F0000904090220000101008032090400000205
:100100005842000007058203200004070502030887
:10011000000412011001000000085E040202000148
:1001200000000001000000070002010000030406B7
:1001300000000000000000000102040810204080C0
:100140000102040810200102040810200404040421
:100150000404040402020202020203030303030371
:1001600000000000230026002900000000002500F8
:1001700028002B0000000000240027002A00112482
:100180001FBECFEFD8E0DEBFCDBF11E0A0E0B1E0F1
:10019000ECEFF3E202C005900D92A832B107D9F757
:1001A00022E0A8E2B1E001C01D92A233B207E1F75C
:1001B0006FD20C94FC1124CFA82FB92F80E090E0CF
:1001C00041E050EA609530E009C02D918227979573
:1001D000879510F084279527305EC8F36F5FA8F3EA
:1001E0000895EADF8D939D930895CF93CFB7CF9372
:1001F000DF93C3954C9BE9F74C9B0BC04C9B09C00C
:100200004C9B07C04C9B05C04C9B03C04C9B01C042
:100210008BC06F93C091F201DD27C750DE4F2F9343
:1002200065E54C9B03C02F916F91E6CF0F931F9311
:100230004F9320E040E15F9309B1047104FB27F97B
:100240003F9350E03BE039C0147140642F77012F99
:100250005F5F1EC0406819B114712F7752501FC0E4
:10026000406409B12F770471D1F15F5F00C023C0F2
:10027000406219B12F77147191F15F5F00C025C002
:1002800004711027515012F45D5F00001150279542
:100290002C3F19B1C8F614710127015027952C3F46
:1002A000C8F64227499309B1047110274F731150C2
:1002B00027952C3FA8F64695469519B1147179F00B
:1002C0000127015027952C3F98F66B5A60F3315067
:1002D00009B1B0F600C011E01CBB002719C03B50AB
:1002E0003195C31BD04011E01CBB0881033C09F1D0
:1002F0000B34F9F02091F0011981110F1213EDCF99
:100300004A81441F093651F10D3211F0013E29F79F
:100310000093F7013F915F914F911F910F912F91A2
:100320006F91CCB3C0FD65CFDF91CF91CFBFCF919F
:1003300018952091F701222369F31091F5011123FB
:10034000E9F53430EAF13093F5012093F101109191
:10035000F2013BE0311B3093F20132C00091F50114
:10036000013064F50AE54F7049F43091050134FD20
:1003700028C000930501C2ECD1E027C0423049F00B
:100380003091CD0134FD1DC00093CD01CEECD1E004
:100390001CC030910F0236FD14C000930F02C0E163
:1003A000D2E013C0052710E000C000000BB91AC04E
:1003B000052710E0221F1DC010E021C04AE502C041
:1003C00032ED432FC4E1D0E032E01AB114615C9AFF
:1003D0000BB11AB954E120E865E320FF05270BB9FA
:1003E000279517951C3FF0F66695B8F7B1F720FFF3
:1003F00005270BB9279517951C3FD0F6279517951C
:1004000017FF052700001C3F0BB9B0F629913A955C
:1004100019F70B7E1091F601110FC651D0400BB9A0
:1004200011F01093F00111E01CBB00611AB11B7EAA
:10043000402F4B7E54E05A95F1F70BB91AB94BB9DE
:1004400069CF1F93CF93DF93162FEA01288124FFF2
:1004500005C0298138E82327298302C02AE528839B
:100460009E012E5F3F4FD901FC01810F91919D9319
:10047000982F9E1B1916D4F3612FC901B2DE1C5FA1
:100480001883DF91CF911F9108954FE052E0D9CFAB
:10049000CF93DF938091F501835087FD91C09091B8
:1004A000F2012091F1012D3209F088C0883009F065
:1004B00085C0CCE0D0E0C91BD109C750DE4F83EC2A
:1004C0008093C2018AE580930501109228018881FA
:1004D000807621F0CE010E94A30A67C09A81109213
:1004E000CB018981811106C01092CC012BEC31E047
:1004F00082E057C0853019F49093F6014FC08630E2
:10050000A9F58B81813041F482E191E09093F4016F
:100510008093F30182E126C0823041F482EF90E0C3
:100520009093F4018093F30180E21CC08330C9F4FE
:10053000911108C08EEE90E09093F4018093F30146
:1005400084E010C0913019F484EC90E004C0923043
:1005500041F48AE990E09093F4018093F3018AE2F8
:1005600001C080E090E4909328011FC0883079F0AA
:10057000893019F49093F80111C08A3059F08B300A
:1005800069F48BE48093CE018093100207C028EFBA
:1005900031E002C02BEC31E081E003C02BEC31E014
:1005A00080E03093F4012093F3019F81911104C006
:1005B0009E81981708F4892F809304011092F50109
:1005C0008091050184FF46C0809104018F3F09F4AA
:1005D00041C0C82F893008F0C8E08C1B809304010B
:1005E0008091C20198E889278093C201CC2331F120
:1005F0002091F3013091F4018091280186FF0BC016
:10060000A3ECB1E0F9018C2F8A0F94919D93319660
:100610008A13FBCF09C0D901E3ECF1E08C2F8E0FD8
:100620009D9191938E13FCCF8FEF8C0F90E00196EC
:10063000820F931F9093F4018093F3016C2F83EC4E
:1006400091E0CFDDCC5FCC3019F08FEF80930401C7
:10065000C093050184E199B1947131F48150D9F7C7
:100660001092F6011092F001DF91CF910895E9E622
:10067000F0E0808182608083E89A8BE48093CE01F1
:10068000809310028AE58093CD0180930F02089534
:100690000E940511A5D0D9D6FECFCF92DF92EF925E
:1006A000FF920F931F93CF93DF9360E086E00E9449
:1006B000321061E086E00E94521060E088E00E9403
:1006C000321061E088E00E94521060E089E00E94F0
:1006D000321061E089E00E94521060E08AE00E94DE
:1006E000321061E08AE00E94521060E08BE00E94CC
:1006F000321061E08BE00E94521060E08CE00E94BA
:10070000321061E08CE00E9452108CE00E9489104F
:10071000892B09F057C086E00E948910892B19F4B3
:10072000C0E1D0E002C0C0E0D0E088E00E948910C3
:10073000892B19F408E010E002C000E010E089E025
:100740000E9489106C018AE00E9489107C018BE074
:100750000E9489109801282B392B2C2B3D2BCC0C77
:10076000DD1CCC0CDD1C2C293D29EE0CFF1C2E2998
:100770003F29C90143E0959587954A95E1F7837034
:100780009927892BD9F02B31310579F03CF42F30A2
:100790003105D9F02731310541F00DC02C3131053B
:1007A00039F02F31310589F006C087E190E00FC0A4
:1007B00084E090E00CC087E090E009C0C901877038
:1007C000992705C08FEF9FEF02C08FE090E0DF9187
:1007D000CF911F910F91FF90EF90DF90CF900895F0
:1007E00081E06DD6D5D6892B39F49FD680E197E28A
:1007F0000E94FB109CD6F6CF0895CFD696D6DCD6B5
:1008000020912B0180FF02C0216001C02E7F209328
:100810002B0120912B0181FF02C0226001C02D7F9E
:1008200020932B0120912B0182FF02C0246001C084
:100830002B7F20932B0120912B0183FF02C0286086
:1008400001C0277F20932B019C0156E03695279508
:100850005A95E1F72170219520932D019C0164E0C8
:10086000369527956A95E1F72170219520932E0101
:100870009C0175E0369527957A95E1F721702195D1
:100880002093310192FB222720F9219520932F01FB
:1008900091FB222720F9219520933001292F2170E7
:1008A00021952093320120912B0193FF02C02062F9
:1008B00001C02F7D20932B0120912B0187FF02C0C7
:1008C000206101C02F7E20932B01817899272091F0
:1008D0002B018138910511F4206801C02F772093F6
:1008E0002B0125D68BCF4DE050E067E070E086E02D
:1008F00090E00E94250D19D680E190E00E94430D02
:1009000020912B0180FF02C0216001C02E7F209327
:100910002B0120912B0181FF02C0226001C02D7F9D
:1009200020932B0120912B0182FF02C0246001C083
:100930002B7F20932B0120912B0183FF02C0286085
:1009400001C0277F20932B019C01E4E03695279579
:10095000EA95E1F72170219520932F019C01F5E0A4
:1009600036952795FA95E1F72170219520932D0171
:100970009C01A6E036952795AA95E1F7217021956F
:10098000209330019C01220F232F221F330B31951E
:100990002170219520932E01292F217021952093DC
:1009A000320191FB222720F921952093310192FBFE
:1009B000222720F921952093330193FB222720F948
:1009C00021952093340120912B0194FF02C02062D5
:1009D00001C02F7D20932B0120912B0195FF02C098
:1009E000206101C02F7E20932B0120912B0196FFC7
:1009F00002C0206401C02F7B20932B0120912B018A
:100A000097FF02C0206801C02F7720932B018FD55C
:100A100072CF47E050E066E070E085E090E00E9431
:100A2000250D83D588E090E00E94430D20912B0195
:100A300084FF02C0216001C02E7F20932B012091F2
:100A40002B0185FF02C0226001C02D7F20932B0166
:100A500020912B0186FF02C0246001C02B7F2093D0
:100A60002B0120912B0187FF02C0286001C0277F46
:100A700020932B019C013695279521702195209379
:100A80002E019C0121703327219520932D01209167
:100A90002B0182FF02C0206201C02F7D20932B0119
:100AA00020912B0183FF02C0206101C02F7E209383
:100AB0002B018C70992720912B010C9711F4206841
:100AC00001C02F7720932B0132D5ABCF47E050E008
:100AD00066E070E085E090E0B8D727D580E190E04F
:100AE000D2D720912B0184FF02C0216001C02E7F4C
:100AF00020932B0120912B0185FF02C0226001C0B1
:100B00002D7F20932B0120912B0186FF02C02460B2
:100B100001C02B7F20932B0120912B0187FF02C066
:100B2000286001C0277F20932B019C01217033276F
:100B3000219520932D01292F2170219520932E019D
:100B40009C01369527952170219520932F0191FBCB
:100B5000222720F921952093300192FB222720F9AA
:100B600021952093330193FB222720F9219520938F
:100B7000340120912B0182FF02C0206201C02F7D31
:100B800020932B0120912B0183FF02C0206101C023
:100B90002F7E20932B018C70992720912B010C978D
:100BA00011F4206801C02F7720932B01C0D495CF7A
:100BB00081E00E941A0E892B39F0B7D480E197E2C8
:100BC0000E94FB10B4D4F4CFDFE7CFEF30E8932ED0
:100BD000ACD40E94FE0D0E94AD0E811111C0109286
:100BE000360110923501109238011092370110929F
:100BF0003A011092390110923C0110923B0178C0E9
:100C000087E090E00E94A80E682F70E080E090E0FE
:100C10001F921F92DF93CF93A12CE0E8BE2ECC242D
:100C2000CA94DC2CE12CF12C8701EA9420E030E01E
:100C3000A9010E944011709336016093350188E04C
:100C400090E00E94A80E682F70E080E090E0CF93C3
:100C5000CF939F921F92AA24AA94AFE7BA2EC12CD9
:100C6000D12C20E030E0A9010E944011709338019E
:100C70006093370185E090E00E94A80E682F70E035
:100C800080E090E01F921F92DF93CF93A12CB0E8F9
:100C9000BB2ECC24CA94DC2C20E030E0A9010E94B9
:100CA000401170933A016093390186E090E00E9410
:100CB000A80E682F70E080E090E0CF93CF939F92D2
:100CC0001F92AA24AA942FE7B22EC12CD12C20E087
:100CD00030E0A9010E94401170933C0160933B01F8
:100CE0008DB79EB740960FB6F8949EBF0FBE8DBFCE
:100CF00080E190E00E949B0E90912B01882311F0DF
:100D0000916001C09E7F90932B0180E490E00E944F
:100D10009B0E90912B01882311F0926001C09D7F62
:100D200090932B0180E890E00E949B0E90912B0104
:100D3000882311F0946001C09B7F90932B0180E287
:100D400090E0F9D790912B01882311F0986001C0B1
:100D5000977F90932B0180E090E8EDD78195809369
:100D60002F0180E090E1E7D781958093300180E00A
:100D700090E4E1D7819580932D0180E090E2DBD76C
:100D8000819580932E0188E090E0D5D790912B013A
:100D9000882311F0906101C09F7E90932B0181E028
:100DA00090E0C9D790912B01882311F0906201C087
:100DB0009F7D90932B0182E090E0BDD790912B0115
:100DC000882311F0906401C09F7B90932B0184E0F5
:100DD00090E0B1D790912B01882311F0906801C069
:100DE0009F7790932B0180E091E0A5D78195809328
:100DF000330180E092E09FD781958093340180E0B9
:100E000094E099D781958093320180E098E093D760
:100E10008195809331018BD3DBCE46D5811107C0FC
:100E200084D380E197E20E94FB1081D3F6CFBFE725
:100E30008B2E99249A94C0E87C2E77D368D5EC0148
:100E4000998180912B0193FF02C0816001C08E7F48
:100E500080932B01998180912B0192FF02C08260C7
:100E600001C08D7F80932B01998180912B0190FF90
:100E700002C0846001C08B7F80932B019981809197
:100E80002B0191FF02C0886001C0877F80932B01F6
:100E9000888183FB882780F9819580932F01888141
:100EA00086958170819580932D01888182FB8827AA
:100EB00080F981958093300188818170819580933C
:100EC0002E01988180912B0194FF02C0806101C0A6
:100ED0008F7E80932B01898186FB882780F98195FD
:100EE00080933301898185FB882780F981958093E0
:100EF00034018981829581708195809331016A8165
:100F000070E080E090E01F921F928F929F92A12C40
:100F100040E8B42ECC24CA94DC2C1FEDE12EF12C39
:100F200000E010E020E230E040E050E00E9440119C
:100F300070933601609335016B81609570E080E0BD
:100F400090E09F929F927F921F92AA24AA94EFE72B
:100F5000BE2EC12CD12C20E230E040E050E00E94B7
:100F6000401170933801609337016C8170E080E02C
:100F700090E01F921F928F929F92A12CF0E8BF2EBB
:100F8000CC24CA94DC2C20E230E040E050E00E9407
:100F9000401170933A01609339016D81609570E062
:100FA00080E090E09F929F927F921F92AA24AA9441
:100FB000AFE7BA2EC12CD12C20E230E040E050E067
:100FC0000E94401170933C0160933B0199812DB7C1
:100FD0003EB7205F3F4F0FB6F8943EBF0FBE2DBF08
:100FE00080912B0193FF05C0988194FF02C0806817
:100FF00001C08F7780932B019AD288E893E10E94F9
:10100000FB101BCF51D4811107C08FD280E197E232
:101010000E94FB108CD2F6CF4FE7442E55245A94F1
:1010200050E8352E812C60E8962E66246A947FE77E
:10103000772E7BD2BED4EC01988180912B0193FF57
:1010400002C0816001C08E7F80932B0198818091C6
:101050002B0192FF02C0826001C08D7F80932B0123
:10106000988180912B0191FF02C0846001C08B7F29
:1010700080932B01988180912B0190FF02C08860A2
:1010800001C0877F80932B01888186FB882780F9A8
:10109000819580932F018881880F880B80932D0183
:1010A000988180912B0194FF02C0806101C08F7EE6
:1010B00080932B01898185FB882780F98195809316
:1010C0003301898182958170819580933401888173
:1010D00085FB882780F98195809331012B8020E85A
:1010E000220E20946A81605870E080E090E01F92A8
:1010F0001F924F925F92A12C10E8B12ECC24CA947B
:10110000DC2C1FEDE12EF12C00E010E020E230E0BD
:1011100040E050E00E944011709336016093350129
:10112000622D70E080E090E05F925F923F921F92AC
:10113000AA24AA943FE7B32EC12CD12C20E230E0A0
:1011400040E050E00E9440117093380160933701F5
:1011500010923A011092390110923C0110923B0119
:1011600089812DB73EB7285F3F4F0FB6F8943EBF39
:101170000FBE2DBF83FF05C070923C0160923B0102
:1011800006C082FF04C090923C0180923B0189819D
:1011900081FF05C090923A018092390106C080FF1C
:1011A00004C070923A0160923901888188719091EF
:1011B0002B01883111F4906801C09F7790932B0127
:1011C000B6D137CF47E050E066E070E085E090E0D0
:1011D0003CD4ABD180E190E056D420912B0182FF2A
:1011E00002C0216001C02E7F20932B0120912B0192
:1011F00094FF02C0226001C02D7F20932B0120911B
:101200002B0181FF02C0246001C02B7F20932B01A2
:1012100020912B0193FF02C0286001C0277F2093FB
:101220002B01292F220F220B20932F019C012170CB
:101230003327219520932D0192FB222720F9219518
:1012400020932E0191FB222720F921952093300134
:1012500020912B0190FF02C0206201C02F7D2093BE
:101260002B0120912B0196FF02C0206101C02F7E2F
:1012700020932B018827917420912B018115914493
:1012800011F4206801C02F7720932B0150D1A1CFFA
:1012900074D54BD17FD520912B0190FF02C02160E6
:1012A00001C02E7F20932B0120912B0191FF02C0C2
:1012B000226001C02D7F20932B0120912B0192FFF2
:1012C00002C0246001C02B7F20932B0120912B01B1
:1012D00093FF02C0286001C0277F20932B019C014F
:1012E000E6E036952795EA95E1F721702195209360
:1012F0002D019C01F4E036952795FA95E1F72170D0
:10130000219520932E019C01A5E036952795AA955D
:10131000E1F721702195209331019C0136952795A5
:10132000369527952170219520932F019C013695A4
:10133000279521702195209330019C01217033273E
:1013400021952093320194FB222720F921952093A7
:1013500033019C0153E0369527955A95E1F72170AA
:1013600021952093340120912B0187FF02C0206139
:1013700001C02F7E20932B018078917020912B014A
:101380008038914011F4206801C02F7720932B0101
:10139000CED07FCF94D5C9D09FD520912B0180FF8F
:1013A00002C0216001C02E7F20932B0120912B01D0
:1013B00082FF02C0226001C02D7F20932B0120916B
:1013C0002B0183FF02C0246001C02B7F20932B01DF
:1013D00020912B0181FF02C0286001C0277F20934C
:1013E0002B019C0164E0369527956A95E1F7217001
:1013F000219520932D019C0175E0369527957A95CE
:10140000E1F72170219520932F0120912B0187FF77
:1014100002C0206101C02F7E20932B0120912B015F
:1014200086FF02C0206201C02F7D20932B01807CAB
:10143000992720912B01803C910511F4206801C06F
:101440002F7720932B0173D0A6CF27D9019689310E
:10145000910570F48C5C9F4FFC018DC744DAD9DA9A
:1014600035DBA6DBDADCCEDDADDE12DF93DFFFCFCE
:10147000C4D984E2E9E2F1E0DF011D928A95E9F73F
:1014800084E180932A0190E190933D0192E490934E
:101490003E0191E0909340019093410192E090933E
:1014A00042018093430186E080934401E5E4F1E04A
:1014B0008FEF8193B1E0ED34FB07D9F70895CF9317
:1014C000DF931F92CDB7DEB790916E009E7F909311
:1014D0006E008983CEDF8981882361F02FE088E167
:1014E00090E00FB6F894A895809360000FBE20930B
:1014F000600008C088E10FB6F894809360001092F5
:1015000060000FBEB4D8549A80E0815041F0A89595
:10151000EFE9FFE03197F1F700C00000F6CF5498F3
:1015200078940F90DF91CF910895A89508958091B8
:101530000F0286FD03C00E944802F9CF64E189E2F0
:1015400091E00C944502FC0180818076803259F450
:1015500081818130D9F489E291E09093F401809304
:10156000F30184E10895803489F48181863071F437
:1015700081E090E090934E0180934D018DE391E0E6
:101580009093F4018093F30180E1089580E0089541
:1015900080914D0190914E01089555985698579815
:1015A00020982198229A23985D9A5E9A5F9A289AA9
:1015B000299A2A9A2B9A0895EF92FF920F931F93DC
:1015C000CF93DF932A9A8EE090E015D689B1829569
:1015D0008695877091E089278170C82F80E0D82F89
:1015E0004E9903C082E090E002C080E090E0C82BFA
:1015F000D92B4F9903C084E090E002C080E090E0D6
:10160000C82BD92B189903C048E050E002C040E035
:1016100050E0C42BD52B199903C020E130E002C063
:1016200020E030E0C22BD32B1B9903C020E230E036
:1016300002C020E030E0C22BD32B2A988EE090E04D
:10164000DAD54F9902C0189B02C0CE0160C0199B29
:1016500025C080E090E08C2B9D2B1B9903C020E8D7
:1016600030E002C020E030E07C01E22AF32A2A9A2E
:101670008EE090E0C0D52A988EE090E0BCD54D99E0
:1016800006C04E9904C04F9902C0189B0AC0C0E022
:10169000D0E09C2F88278E299F2939C080E490E0D4
:1016A000DACF2A9A8EE090E0A6D589B18295869508
:1016B000877091E08927082F017010E04E9B24C0AD
:1016C00020E030E0E901C02BD12B4F9903C084E02A
:1016D00090E002C080E090E0C82BD92B189903C09D
:1016E00048E050E002C040E050E0C42BD52B2A98DF
:1016F0008EE090E080D52A9A8EE090E07CD52A9802
:1017000080ED97E078D5C5CF22E030E0DBCFDF91E8
:10171000CF911F910F91FF90EF900895559A20E877
:10172000FC01408142235D9830E009F440C0000094
:101730000000000000000000000000005D9A3595E8
:101740002795211112C00196615000000000000091
:101750000000000000000000000000000000000089
:1017600000000000000020E814C00000000000009D
:101770000000000000000000000000000000000069
:101780000000000000000000000000000000000059
:101790000000000000000000000000000000000049
:1017A00000000000000000000000000040C0000039
:1017B0000000000000000000000000000000000029
:1017C00000000000000035952795211112C00196F8
:1017D0006150000000000000000000000000000058
:1017E000000000000000000000000000000020E8F1
:1017F00013C0000000000000000000000000000016
:1018000000000000000000000000000000000000D8
:1018100000000000000000005D9A000000000000D1
:101820000000000000000000000000000000611146
:1018300077CF000000005D9800000000000000006D
:101840000000000000000000000000000000000098
:10185000000000005D9A089555985D9AEBE5F1E06F
:101860008E0F4D99FECF0000000000000000000028
:101870000000000000000000000000000000000068
:101880000000000000000000000000000000000058
:1018900000000000000099B1907291938E1719F02A
:1018A0004D9BFECFDECF08951F93CF93DF931F9202
:1018B000CDB7DEB71982EBE5F1E0119281E0EB39AB
:1018C000F807D9F7E3E5F1E0119281E0EB35F8078D
:1018D000D9F710924F0110925001109251011092BD
:1018E0005201F89461E0CE01019618DF55985D9A97
:1018F00010E44D9B02C01150E1F7789484EF91E021
:101900007AD4812F0F90DF91CF911F9108951F936B
:10191000CF93DF9300D01F92CDB7DEB780E48983E9
:1019200083E08A831B82F89463E0CE010196F6DEA1
:1019300080E492DF7894E3E5F1E04BE551E087E065
:1019400090E061E070E020E030E0DA01A20FB31F28
:10195000AC91AA2351F01081DB01082E01C0AA0F1F
:101960000A94EAF71A2B10830AC0DB01082E01C083
:10197000AA0F0A94EAF7A095B081BA23B083019721
:1019800097FF02C087E090E02F5F3F4F283031057E
:10199000E1F63196485F5F4F21E0EB35F20799F6AB
:1019A00083E591E00F900F900F90DF91CF911F9101
:1019B00008951F93CF93DF931F92CDB7DEB781E0D9
:1019C0008983F89461E0CE010196A8DE80E244DFCD
:1019D0007894EFE4F1E04BE551E087E090E061E0DE
:1019E00070E020E030E0DA01A20FB31FAC91AA232F
:1019F00051F01081DB01082E01C0AA0F0A94EAF70A
:101A00001A2B10830AC0DB01082E01C0AA0F0A940A
:101A1000EAF7A095B081BA23B083019797FF02C07F
:101A200087E090E02F5F3F4F28303105E1F6319697
:101A3000485F5F4F21E0E335F20799F68FE491E0CC
:101A40000F90DF91CF911F910895CF93DF938093F3
:101A50009F019093A00170939E0160939D0150930C
:101A60009C0140939B0161E0FDD261E080919D016A
:101A7000F9D2CBE9D1E060E08881F4D261E08881DD
:101A8000DF91CF910FC3EF92FF920F931F93CF93EC
:101A9000DF937C0160E080919D0104D360E0809140
:101AA0009F0100D361E080919D01FCD281E090E034
:101AB000A2D360E080919D01F5D280919B0129D352
:101AC0008C01C1E0D0E0CE15DF05C4F461E0809167
:101AD0009F01E8D281E090E08ED360E080919F0189
:101AE000E1D280919B0115D30C2E02C0880F991F63
:101AF0000A94E2F7082B192B2196E5CFC8018095AF
:101B00009095DF91CF911F910F91FF90EF900895E5
:101B1000CF92DF92EF92FF920F931F93CF93DF93B9
:101B2000C0E0D0E0D12C082F10E0EE24E394F12C9B
:101B30002898CC2EA8010C2E02C0559547950A94E2
:101B4000E2F740FF02C05E9A01C05E9884E190E037
:101B500052D3289A4D9B07C097010C2C01C0220F2D
:101B60000A94EAF7D22A84E190E045D32196C8305E
:101B7000D105F1F6289A83E090E03DD38D2DDF91D9
:101B8000CF911F910F91FF90EF90DF90CF9008952C
:101B9000EF92FF920F931F93CF93DF93182FF92E9D
:101BA000062F8091A201882309F0F8945F985E9A2D
:101BB000289A86E090E01FD3E12EC12FDF2D8C2FD5
:101BC0008E19801720F48881A3DF8993F8CF5F9A5C
:101BD0008091A201882309F078942091060188EE73
:101BE00093E0AC01249FC001259F900D1124DF914B
:101BF000CF911F910F91FF90EF90FDC281E08093F4
:101C0000A30182E48093A4012091060188EE93E071
:101C1000AC01249FC001259F900D1124ECD2E5EA70
:101C2000F1E0119251E0E83BF507D9F765E183EA6D
:101C300091E0AECFFF920F931F93CF93DF93CDB779
:101C4000DEB7A0970FB6F894DEBF0FBECDBF80936E
:101C5000A20155985D9A209A579A569A289A5E9AA8
:101C6000CDDF8091A401813429F0833719F08937C1
:101C700009F050C081E08093060103E095E0F92E61
:101C800019E0E7E0F1E0DE015C968F2D01900D9206
:101C90008A95E1F765E0CE014C967ADFECE0F1E061
:101CA000DE015396812F01900D928A95E1F769E04C
:101CB000CE0143966DDF8E898093B801E5E1F1E0B6
:101CC000DE011A96812F01900D928A95E1F769E065
:101CD000CE010A965DDFEEE1F1E0DE011196812F83
:101CE00001900D928A95E1F769E0CE01019650DFEF
:101CF00085DF8091A401833721F481E08093A101E5
:101D00000CC0809106018F5F80930601015009F09D
:101D1000B8CF03C081E090E002C080E090E0A096E0
:101D20000FB6F894DEBF0FBECDBFDF91CF911F91EC
:101D30000F91FF9008952091A6013091A701209561
:101D400030952823392381E0232B09F480E008957E
:101D50008D559E4FFC01808108958091B80183309C
:101D600041F09091A101911104C0813021F482E0F1
:101D7000089581E0089580E0089555985698229836
:101D80002398579A219A5D9A5E9A2A9A2B9A5F9A7B
:101D9000299A08950F931F93CF93DF935F9A299AFF
:101DA00084E090E028D21A9903C000E010E102C05C
:101DB00000E010E05F98299884E090E01CD289B19F
:101DC000829586958695837091E089278170C82FCA
:101DD00080E0D82FC02BD12B4D9903C042E050E0BA
:101DE00002C040E050E0C42BD52B1B9903C044E057
:101DF00050E002C040E050E04C2B5D2B1A9903C02C
:101E000028E030E002C020E030E0EA01C22BD32B12
:101E10005F9A299884E090E0EED14E9903C080E16A
:101E200090E002C080E090E0C82BD92B4D9903C010
:101E300040E250E002C040E050E0C42BD52B1B999B
:101E400003C020E430E002C020E030E0C22BD32BFE
:101E50001A9903C080E890E002C080E090E0C82BAF
:101E6000D92B5F98299A84E090E0C5D14E9903C0A0
:101E700040E051E002C040E050E04C2B5D2B4D991A
:101E800003C020E032E002C020E030E0242B352BFC
:101E90001B9903C080E094E002C080E090E0822BB8
:101EA000932B1A9903C020E038E002C020E030E014
:101EB000822B932BDF91CF911F910F91089555980D
:101EC0005D9A57985F9A2098289A2198299A229A81
:101ED0002A9A239A2B980895DF92EF92FF920F93FC
:101EE0001F93CF93DF932A9A2B9882E0E82EF12C50
:101EF000C0E0D0E0DD24D3942B9881E090E07BD14A
:101F00004D993DC04F993BC0189939C0199937C0B8
:101F10002A9881E090E06FD14D9B2EC080E090E048
:101F2000C82BD92B4F9903C020E032E002C020E03B
:101F300030E0C22BD32B189903C020E034E002C05C
:101F400020E030E0C22BD32B199903C020E038E009
:101F500002C020E030E0C22BD32B2A9A2B9A81E0DA
:101F6000E81AF10849F6CE01DF91CF911F910F9148
:101F7000FF90EF90DF90089580E091E0D1CF89B19C
:101F80008295869587708D25082F017010E00C2BA7
:101F90001D2B4F9B3BC080E090E0E801C82BD92B64
:101FA000189903C024E030E002C020E030E0C22BEA
:101FB000D32B199903C028E030E002C020E030E0C4
:101FC000C22BD32B2A9881E090E015D14D9903C004
:101FD00060E170E002C060E070E0C62BD72B4F9943
:101FE00003C040E250E002C040E050E0C42BD52BDB
:101FF000189903C020E430E002C020E030E0C22B9A
:10200000D32B1999A6CF20E830E0A5CF82E090E04D
:10201000C4CF833081F028F4813099F08230A1F070
:1020200008958630A9F08730B9F08430D1F48091DA
:1020300080008F7D03C0809180008F778093800027
:10204000089584B58F7702C084B58F7D84BD0895CF
:102050008091B0008F7703C08091B0008F7D809316
:10206000B000089590E0FC01E85CFE4F2491FC0173
:10207000E45BFE4FE491EE23A1F0F0E0EE0FFF1FD2
:10208000EC58FE4FA591B4919FB7611105C0F8942B
:102090008C912095822303C0F8948C91822B8C9391
:1020A0009FBF08950F931F93CF93DF931F92CDB7D8
:1020B000DEB7282F30E0F901EC5DFE4F8491F90185
:1020C000E85CFE4F1491F901E45BFE4F049100239C
:1020D000D1F0882319F069839CDF6981E02FF0E05B
:1020E000EE0FFF1FE659FE4FA591B4919FB7611106
:1020F00005C0F8948C911095812303C0F8948C91BD
:10210000812B8C939FBF0F90DF91CF911F910F91E7
:102110000895CF93DF93282F30E0F901EC5DFE4F57
:102120008491F901E85CFE4FD491F901E45BFE4F24
:10213000C491CC2389F081116CDFEC2FF0E0EE0F1D
:10214000FF1FE05AFE4FA591B4912C912D2381E001
:1021500090E021F480E002C080E090E0DF91CF9138
:1021600008951F920F920FB60F9211242F933F9351
:102170008F939F93AF93BF938091BA019091BB01CE
:10218000A091BC01B091BD013091B90123E0230FB2
:102190002D3720F40196A11DB11D05C026E8230F9F
:1021A0000296A11DB11D2093B9018093BA019093AD
:1021B000BB01A093BC01B093BD018091BE01909181
:1021C000BF01A091C001B091C1010196A11DB11D37
:1021D0008093BE019093BF01A093C001B093C10151
:1021E000BF91AF919F918F913F912F910F900FBE13
:1021F0000F901F901895019739F0880F991F880F3D
:10220000991F02970197F1F70895789484B5826039
:1022100084BD84B5816084BD85B5826085BD85B58A
:10222000816085BDEEE6F0E0808181608083E1E839
:10223000F0E0108280818260808380818160808371
:10224000E0E8F0E0808181608083E1EBF0E0808174
:1022500084608083E0EBF0E0808181608083EAE746
:10226000F0E08081846080838081826080838081CF
:10227000816080838081806880831092C10008958E
:102280004F925F926F927F92AF92BF92CF92DF9206
:10229000EF92FF920F931F93CF93DF93CDB7DEB7EB
:1022A00029013A01621773078407950754F0DC018E
:1022B000CB01E816F9060A071B072CF4D801C70161
:1022C00002C0DA01C9019C01AD0124193509460992
:1022D000570989899A89AB89BC89BC01CD016A19E2
:1022E0007B098C099D091CD0A80197012419350987
:1022F0004609570924D02A0D3B1D4C1D5D1DCA01FE
:10230000B901DF91CF911F910F91FF90EF90DF9076
:10231000CF90BF90AF907F906F905F904F90089557
:10232000DB018F939F932DD0BF91AF91A29F800D22
:10233000911DA39F900DB29F900D11240895052E1D
:1023400097FB16F400940FD057FD05D024D007FC5E
:1023500002D046F408C050954095309521953F4FE6
:102360004F4F5F4F089590958095709561957F4F81
:102370008F4F9F4F0895EE0FFF1F0590F491E02DB2
:1023800009942BD0A59F900DB49F900DA49F800D14
:10239000911D11240895A1E21A2EAA1BBB1BFD0159
:1023A0000DC0AA1FBB1FEE1FFF1FA217B307E40734
:1023B000F50720F0A21BB30BE40BF50B661F771F8C
:1023C000881F991F1A9469F760957095809590956C
:1023D0009B01AC01BD01CF010895A29FB001B39F45
:1023E000C001A39F700D811D1124911DB29F700D1E
:0C23F000811D1124911D0895F894FFCF69
:1023FC0001000000FF5A0101430001000145005A91
:10240C005A5A5A5A5A014400010300000000014371
:08241C0000005A5A5A5A5A00F6
:00000001FF
